 jpeg

 Timestamp is 68fa8ffe (Thu Oct 23 20:28:46 2025)

 Preferred load address is 10000000

 Start         Length     Name                   Class
 0001:00000000 0001dff9H .text$mn                CODE
 0002:00000000 000000b4H .idata$5                DATA
 0002:000000b4 00000008H .00cfg                  DATA
 0002:000000bc 00000004H .CRT$XCA                DATA
 0002:000000c0 00000004H .CRT$XCZ                DATA
 0002:000000c4 00000004H .CRT$XIA                DATA
 0002:000000c8 00000004H .CRT$XIZ                DATA
 0002:000000cc 00000004H .CRT$XPA                DATA
 0002:000000d0 00000004H .CRT$XPZ                DATA
 0002:000000d4 00000004H .CRT$XTA                DATA
 0002:000000d8 00000008H .CRT$XTZ                DATA
 0002:000000dc 00000000H .gfids$y                DATA
 0002:000000e0 000024e0H .rdata                  DATA
 0002:000025c0 00000000H .rdata$CastGuardVftablesA DATA
 0002:000025c0 00000000H .rdata$CastGuardVftablesC DATA
 0002:000025c0 00000004H .rdata$sxdata           DATA
 0002:000025c4 00000064H .rdata$voltmd           DATA
 0002:00002628 000002e8H .rdata$zzzdbg           DATA
 0002:00002910 00000004H .rtc$IAA                DATA
 0002:00002914 00000004H .rtc$IZZ                DATA
 0002:00002918 00000004H .rtc$TAA                DATA
 0002:0000291c 00000004H .rtc$TZZ                DATA
 0002:00002920 00000090H .xdata$x                DATA
 0002:000029b0 00000634H .edata                  DATA
 0002:00002fe4 0000008cH .idata$2                DATA
 0002:00003070 00000014H .idata$3                DATA
 0002:00003084 000000b4H .idata$4                DATA
 0002:00003138 000003b0H .idata$6                DATA
 0003:00000000 00000028H .data                   DATA
 0003:00000028 000003d4H .bss                    DATA
 0004:00000000 00000060H .rsrc$01                DATA
 0004:00000060 00000330H .rsrc$02                DATA

  Address         Publics by Value              Rva+Base       Lib:Object

 0000:00000000       ___AbsoluteZero            00000000     <absolute>
 0000:00000000       ___arm64x_extra_rfe_table  00000000     <absolute>
 0000:00000000       ___arm64x_extra_rfe_table_size 00000000     <absolute>
 0000:00000000       ___arm64x_native_entrypoint 00000000     <absolute>
 0000:00000000       ___arm64x_redirection_metadata 00000000     <absolute>
 0000:00000000       ___arm64x_redirection_metadata_count 00000000     <absolute>
 0000:00000000       ___dynamic_value_reloc_table 00000000     <absolute>
 0000:00000000       ___enclave_config          00000000     <absolute>
 0000:00000000       ___guard_check_icall_a64n_fptr 00000000     <absolute>
 0000:00000000       ___guard_eh_cont_count     00000000     <absolute>
 0000:00000000       ___guard_eh_cont_table     00000000     <absolute>
 0000:00000000       ___guard_fids_count        00000000     <absolute>
 0000:00000000       ___guard_fids_table        00000000     <absolute>
 0000:00000000       ___guard_iat_count         00000000     <absolute>
 0000:00000000       ___guard_iat_table         00000000     <absolute>
 0000:00000000       ___guard_longjmp_count     00000000     <absolute>
 0000:00000000       ___guard_longjmp_table     00000000     <absolute>
 0000:00000000       ___hybrid_auxiliary_delayload_iat 00000000     <absolute>
 0000:00000000       ___hybrid_auxiliary_delayload_iat_copy 00000000     <absolute>
 0000:00000000       ___hybrid_auxiliary_iat    00000000     <absolute>
 0000:00000000       ___hybrid_auxiliary_iat_copy 00000000     <absolute>
 0000:00000000       ___hybrid_code_map         00000000     <absolute>
 0000:00000000       ___hybrid_code_map_count   00000000     <absolute>
 0000:00000000       ___hybrid_image_info_bitfield 00000000     <absolute>
 0000:00000000       ___x64_code_ranges_to_entry_points 00000000     <absolute>
 0000:00000000       ___x64_code_ranges_to_entry_points_count 00000000     <absolute>
 0000:00000001       ___safe_se_handler_count   00000001     <absolute>
 0000:00000100       ___guard_flags             00000100     <absolute>
 0000:00000000       ___ImageBase               10000000     <linker-defined>
 0001:000000c0       _Java_com_sun_imageio_plugins_jpeg_JPEGImageReader_abortRead@16 100010c0 f   imageioJPEG.obj
 0001:000000f0       _Java_com_sun_imageio_plugins_jpeg_JPEGImageReader_disposeReader@16 100010f0 f   imageioJPEG.obj
 0001:000000f0       _Java_com_sun_imageio_plugins_jpeg_JPEGImageWriter_disposeWriter@16 100010f0 f   imageioJPEG.obj
 0001:00000140       _Java_com_sun_imageio_plugins_jpeg_JPEGImageReader_initJPEGImageReader@8 10001140 f   imageioJPEG.obj
 0001:00000380       _Java_com_sun_imageio_plugins_jpeg_JPEGImageReader_initReaderIDs@20 10001380 f   imageioJPEG.obj
 0001:00000550       _Java_com_sun_imageio_plugins_jpeg_JPEGImageReader_readImage@84 10001550 f   imageioJPEG.obj
 0001:00001300       _Java_com_sun_imageio_plugins_jpeg_JPEGImageReader_readImageHeader@24 10002300 f   imageioJPEG.obj
 0001:00001770       _Java_com_sun_imageio_plugins_jpeg_JPEGImageReader_resetLibraryState@16 10002770 f   imageioJPEG.obj
 0001:000017a0       _Java_com_sun_imageio_plugins_jpeg_JPEGImageReader_resetReader@16 100027a0 f   imageioJPEG.obj
 0001:00001830       _Java_com_sun_imageio_plugins_jpeg_JPEGImageReader_setOutColorSpace@20 10002830 f   imageioJPEG.obj
 0001:00001860       _Java_com_sun_imageio_plugins_jpeg_JPEGImageReader_setSource@16 10002860 f   imageioJPEG.obj
 0001:000018b0       _Java_com_sun_imageio_plugins_jpeg_JPEGImageWriter_abortWrite@16 100028b0 f   imageioJPEG.obj
 0001:000018e0       _Java_com_sun_imageio_plugins_jpeg_JPEGImageWriter_initJPEGImageWriter@8 100028e0 f   imageioJPEG.obj
 0001:00001af0       _Java_com_sun_imageio_plugins_jpeg_JPEGImageWriter_initWriterIDs@16 10002af0 f   imageioJPEG.obj
 0001:00001c10       _Java_com_sun_imageio_plugins_jpeg_JPEGImageWriter_resetWriter@16 10002c10 f   imageioJPEG.obj
 0001:00001c60       _Java_com_sun_imageio_plugins_jpeg_JPEGImageWriter_setDest@16 10002c60 f   imageioJPEG.obj
 0001:00001cb0       _Java_com_sun_imageio_plugins_jpeg_JPEGImageWriter_writeImage@116 10002cb0 f   imageioJPEG.obj
 0001:000028d0       _Java_com_sun_imageio_plugins_jpeg_JPEGImageWriter_writeTables@28 100038d0 f   imageioJPEG.obj
 0001:00002e90       _imageio_fill_input_buffer 10003e90 f   imageioJPEG.obj
 0001:00003150       _imageio_init_source       10004150 f   imageioJPEG.obj
 0001:00003150       _sun_jpeg_init_source      10004150 f   jpegdecoder.obj
 0001:00003330       _imageio_skip_input_data   10004330 f   imageioJPEG.obj
 0001:00003660       _imageio_term_source       10004660 f   imageioJPEG.obj
 0001:000038c0       _read_icc_profile          100048c0 f   imageioJPEG.obj
 0001:000040b0       _jCreaCompress             100050b0 f   jcapimin.obj
 0001:000041c0       _jFinCompress              100051c0 f   jcapimin.obj
 0001:000042d0       _jSuppressTables           100052d0 f   jcapimin.obj
 0001:00004380       _jWrtTables                10005380 f   jcapimin.obj
 0001:000043e0       _jStrtCompress             100053e0 f   jcapistd.obj
 0001:00004460       _jWrtScanlines             10005460 f   jcapistd.obj
 0001:00004c10       _jICCoefC                  10005c10 f   jccoefct.obj
 0001:00004ff0       _jICColor                  10005ff0 f   jccolor.obj
 0001:000052c0       @_guard_check_icall_nop@4  100062c0 f   MSVCRT:guard_support.obj
 0001:000052c0       _jMemTerm                  100062c0 f   jmemnobs.obj
 0001:000052c0       _sun_jpeg_term_source      100062c0 f   jpegdecoder.obj
 0001:000062a0       _jIFDCT                    100072a0 f   jcdctmgr.obj
 0001:00007210       _jGenOptTbl                10008210 f   jchuff.obj
 0001:00007460       _jIHEncoder                10008460 f   jchuff.obj
 0001:00007500       _jMkCDerived               10008500 f   jchuff.obj
 0001:000078c0       _jICompress                100088c0 f   jcinit.obj
 0001:00007980       _jICMainC                  10008980 f   jcmainct.obj
 0001:00008650       _jIMWriter                 10009650 f   jcmarker.obj
 0001:00008cd0       _jICMaster                 10009cd0 f   jcmaster.obj
 0001:000096c0       _jAbort                    1000a6c0 f   jcomapi.obj
 0001:00009700       _jAlcHTable                1000a700 f   jcomapi.obj
 0001:00009730       _jAlcQTable                1000a730 f   jcomapi.obj
 0001:00009760       _jDestroy                  1000a760 f   jcomapi.obj
 0001:00009930       _jAddQuantTable            1000a930 f   jcparam.obj
 0001:00009a10       _jSetColorspace            1000aa10 f   jcparam.obj
 0001:00009dd0       _jSetDefaults              1000add0 f   jcparam.obj
 0001:00009fb0       _jSimProgress              1000afb0 f   jcparam.obj
 0001:0000aea0       _jIPHEncoder               1000bea0 f   jcphuff.obj
 0001:0000b0c0       _jICPrepC                  1000c0c0 f   jcprepct.obj
 0001:0000bf10       _jIDownsampler             1000cf10 f   jcsample.obj
 0001:0000c2e0       _jAbrtDecompress           1000d2e0 f   jdapimin.obj
 0001:0000c2f0       _jConsumeInput             1000d2f0 f   jdapimin.obj
 0001:0000c3b0       _jCreaDecompress           1000d3b0 f   jdapimin.obj
 0001:0000c4f0       _jDestDecompress           1000d4f0 f   jdapimin.obj
 0001:0000c500       _jFinDecompress            1000d500 f   jdapimin.obj
 0001:0000c5d0       _jHasMultScn               1000d5d0 f   jdapimin.obj
 0001:0000c610       _jInComplete               1000d610 f   jdapimin.obj
 0001:0000c650       _jReadHeader               1000d650 f   jdapimin.obj
 0001:0000c780       _jFinOutput                1000d780 f   jdapistd.obj
 0001:0000c820       _jReadScanlines            1000d820 f   jdapistd.obj
 0001:0000c8c0       _jStrtDecompress           1000d8c0 f   jdapistd.obj
 0001:0000c9b0       _jStrtOutput               1000d9b0 f   jdapistd.obj
 0001:0000d800       ___scrt_stub_for_is_c_termination_complete 1000e800 f   MSVCRT:ucrt_stubs.obj
 0001:0000d800       __is_c_termination_complete 1000e800 f   MSVCRT:ucrt_stubs.obj
 0001:0000d800       _jMemInit                  1000e800 f   jmemnobs.obj
 0001:0000d810       _jIDCoefC                  1000e810 f   jdcoefct.obj
 0001:0000dd20       _jIDColor                  1000ed20 f   jdcolor.obj
 0001:0000e220       _jIIDCT                    1000f220 f   jddctmgr.obj
 0001:0000ebf0       _jFilBitBuf                1000fbf0 f   jdhuff.obj
 0001:0000ed10       _jHufDecode                1000fd10 f   jdhuff.obj
 0001:0000edf0       _jIHDecoder                1000fdf0 f   jdhuff.obj
 0001:0000ee60       _jMkDDerived               1000fe60 f   jdhuff.obj
 0001:0000f580       _jIInCtlr                  10010580 f   jdinput.obj
 0001:0000f8a0       _jIDMainC                  100108a0 f   jdmainct.obj
 0001:000110b0       _jIMReader                 100120b0 f   jdmarker.obj
 0001:00011170       _jResyncRestart            10012170 f   jdmarker.obj
 0001:00011280       _jSaveMarkers              10012280 f   jdmarker.obj
 0001:00011dc0       _jCalcDimensions           10012dc0 f   jdmaster.obj
 0001:00012060       _jIDMaster                 10013060 f   jdmaster.obj
 0001:00012910       _jIMUpsampler              10013910 f   jdmerge.obj
 0001:000134d0       _jIPHDecoder               100144d0 f   jdphuff.obj
 0001:00013860       _jIDPostC                  10014860 f   jdpostct.obj
 0001:00013fc0       _jIUpsampler               10014fc0 f   jdsample.obj
 0001:000142d0       ___local_stdio_printf_options 100152d0 f i jerror.obj
 0001:000143f0       _fprintf                   100153f0 f i jerror.obj
 0001:00014420       _jStdError                 10015420 f   jerror.obj
 0001:00014510       _jFDfloat                  10015510 f   jfdctflt.obj
 0001:00015ae0       _jFDifast                  10016ae0 f   jfdctfst.obj
 0001:00016a50       _jFDislow                  10017a50 f   jfdctint.obj
 0001:00017fb0       _jRDfloat                  10018fb0 f   jidctflt.obj
 0001:00018470       _jRDifast                  10019470 f   jidctfst.obj
 0001:00018870       _jRDislow                  10019870 f   jidctint.obj
 0001:00018d60       _jRD1x1                    10019d60 f   jidctred.obj
 0001:00018da0       _jRD2x2                    10019da0 f   jidctred.obj
 0001:00018ff0       _jRD4x4                    10019ff0 f   jidctred.obj
 0001:00019310       ___local_stdio_scanf_options 1001a310 f i jmemmgr.obj
 0001:00019b90       _jIMemMgr                  1001ab90 f   jmemmgr.obj
 0001:0001a0a0       _sscanf                    1001b0a0 f i jmemmgr.obj
 0001:0001a0d0       _jFreeLarge                1001b0d0 f   jmemnobs.obj
 0001:0001a0d0       _jFreeSmall                1001b0d0 f   jmemnobs.obj
 0001:0001a0e0       _jGetLarge                 1001b0e0 f   jmemnobs.obj
 0001:0001a0e0       _jGetSmall                 1001b0e0 f   jmemnobs.obj
 0001:0001a0f0       _jMemAvail                 1001b0f0 f   jmemnobs.obj
 0001:0001a110       _jOpenBackStore            1001b110 f   jmemnobs.obj
 0001:0001a1b0       _JNI_OnLoad@8              1001b1b0 f   jpegdecoder.obj
 0001:0001a1d0       _Java_sun_awt_image_JPEGImageDecoder_initIDs@12 1001b1d0 f   jpegdecoder.obj
 0001:0001a280       _Java_sun_awt_image_JPEGImageDecoder_readImage@16 1001b280 f   jpegdecoder.obj
 0001:0001ab10       _sun_jpeg_fill_input_buffer 1001bb10 f   jpegdecoder.obj
 0001:0001ac00       _sun_jpeg_fill_suspended_buffer 1001bc00 f   jpegdecoder.obj
 0001:0001ad90       _sun_jpeg_skip_input_data  1001bd90 f   jpegdecoder.obj
 0001:0001b420       _jI1Quant                  1001c420 f   jquant1.obj
 0001:0001bfd0       _jI2Quant                  1001cfd0 f   jquant2.obj
 0001:0001d140       _jCopyBlocks               1001e140 f   jutils.obj
 0001:0001d160       _jCopySamples              1001e160 f   jutils.obj
 0001:0001d1b0       _jDivRound                 1001e1b0 f   jutils.obj
 0001:0001d1c0       _jRound                    1001e1c0 f   jutils.obj
 0001:0001d1e0       _jZeroFar                  1001e1e0 f   jutils.obj
 0001:0001d1f3       _JNU_ThrowByName@12        1001e1f3 f   java:java.dll
 0001:0001d1f9       _JNU_ThrowNullPointerException@8 1001e1f9 f   java:java.dll
 0001:0001d1ff       _JNU_GetEnv@8              1001e1ff f   java:java.dll
 0001:0001d205       _jio_snprintf              1001e205 f   java:java.dll
 0001:0001d20b       @__security_check_cookie@4 1001e20b f   MSVCRT:secchk.obj
 0001:0001d219       ___isa_available_init      1001e219 f   MSVCRT:cpu_disp.obj
 0001:0001d3ed       ___raise_securityfailure   1001e3ed f   MSVCRT:gs_report.obj
 0001:0001d415       ___report_gsfailure        1001e415 f   MSVCRT:gs_report.obj
 0001:0001d50f       ___report_rangecheckfailure 1001e50f f   MSVCRT:gs_report.obj
 0001:0001d51b       ___report_securityfailure  1001e51b f   MSVCRT:gs_report.obj
 0001:0001d92a       __DllMainCRTStartup@12     1001e92a f   MSVCRT:dll_dllmain.obj
 0001:0001d99a       ___security_init_cookie    1001e99a f   MSVCRT:gs_support.obj
 0001:0001d9e5       _DllMain@12                1001e9e5 f   MSVCRT:dll_dllmain_stub.obj
 0001:0001da07       ?__scrt_initialize_type_info@@YAXXZ 1001ea07 f   MSVCRT:tncleanup.obj
 0001:0001da13       ?__scrt_uninitialize_type_info@@YAXXZ 1001ea13 f   MSVCRT:tncleanup.obj
 0001:0001da1f       ___scrt_initialize_default_local_stdio_options 1001ea1f f   MSVCRT:default_local_stdio_options.obj
 0001:0001da80       ___scrt_acquire_startup_lock 1001ea80 f   MSVCRT:utility.obj
 0001:0001dab2       ___scrt_dllmain_after_initialize_c 1001eab2 f   MSVCRT:utility.obj
 0001:0001dadd       ___scrt_dllmain_before_initialize_c 1001eadd f   MSVCRT:utility.obj
 0001:0001daeb       ___scrt_dllmain_crt_thread_attach 1001eaeb f   MSVCRT:utility.obj
 0001:0001db0a       ___scrt_dllmain_crt_thread_detach 1001eb0a f   MSVCRT:utility.obj
 0001:0001db17       ___scrt_dllmain_exception_filter 1001eb17 f   MSVCRT:utility.obj
 0001:0001db4b       ___scrt_dllmain_uninitialize_c 1001eb4b f   MSVCRT:utility.obj
 0001:0001db6e       ___scrt_dllmain_uninitialize_critical 1001eb6e f   MSVCRT:utility.obj
 0001:0001db7b       ___scrt_initialize_crt     1001eb7b f   MSVCRT:utility.obj
 0001:0001dbb4       ___scrt_initialize_onexit_tables 1001ebb4 f   MSVCRT:utility.obj
 0001:0001dc3b       ___scrt_is_nonwritable_in_current_image 1001ec3b f   MSVCRT:utility.obj
 0001:0001dccf       ___scrt_release_startup_lock 1001eccf f   MSVCRT:utility.obj
 0001:0001dcec       ___scrt_uninitialize_crt   1001ecec f   MSVCRT:utility.obj
 0001:0001dd14       ___scrt_get_dyn_tls_init_callback 1001ed14 f   MSVCRT:dyn_tls_init.obj
 0001:0001dd1a       ___scrt_fastfail           1001ed1a f   MSVCRT:utility_desktop.obj
 0001:0001de35       __crt_debugger_hook        1001ee35 f   MSVCRT:utility_desktop.obj
 0001:0001de3d       __RTC_Initialize           1001ee3d f   MSVCRT:initsect.obj
 0001:0001de69       __RTC_Terminate            1001ee69 f   MSVCRT:initsect.obj
 0001:0001dea0       __SEH_prolog4              1001eea0 f   MSVCRT:sehprolg4.obj
 0001:0001dee5       __except_handler4          1001eee5 f   MSVCRT:chandler4gs.obj
 0001:0001df14       __get_startup_argv_mode    1001ef14 f   MSVCRT:argv_mode.obj
 0001:0001df18       ___scrt_is_ucrt_dll_in_use 1001ef18 f   MSVCRT:ucrt_detection.obj
 0001:0001df24       _longjmp                   1001ef24 f   vcruntime:VCRUNTIME140.dll
 0001:0001df2a       __setjmp3                  1001ef2a f   vcruntime:VCRUNTIME140.dll
 0001:0001df30       _memcpy                    1001ef30 f   vcruntime:VCRUNTIME140.dll
 0001:0001df36       _memset                    1001ef36 f   vcruntime:VCRUNTIME140.dll
 0001:0001df3c       _memmove                   1001ef3c f   vcruntime:VCRUNTIME140.dll
 0001:0001df42       ___std_type_info_destroy_list 1001ef42 f   vcruntime:VCRUNTIME140.dll
 0001:0001df48       __except_handler4_common   1001ef48 f   vcruntime:VCRUNTIME140.dll
 0001:0001df4e       __initterm                 1001ef4e f   ucrt:api-ms-win-crt-runtime-l1-1-0.dll
 0001:0001df54       __initterm_e               1001ef54 f   ucrt:api-ms-win-crt-runtime-l1-1-0.dll
 0001:0001df5a       __seh_filter_dll           1001ef5a f   ucrt:api-ms-win-crt-runtime-l1-1-0.dll
 0001:0001df60       __configure_narrow_argv    1001ef60 f   ucrt:api-ms-win-crt-runtime-l1-1-0.dll
 0001:0001df66       __initialize_narrow_environment 1001ef66 f   ucrt:api-ms-win-crt-runtime-l1-1-0.dll
 0001:0001df6c       __initialize_onexit_table  1001ef6c f   ucrt:api-ms-win-crt-runtime-l1-1-0.dll
 0001:0001df72       __execute_onexit_table     1001ef72 f   ucrt:api-ms-win-crt-runtime-l1-1-0.dll
 0001:0001df78       __cexit                    1001ef78 f   ucrt:api-ms-win-crt-runtime-l1-1-0.dll
 0001:0001df7e       ___acrt_initialize         1001ef7e f   MSVCRT:ucrt_stubs.obj
 0001:0001df7e       ___acrt_thread_attach      1001ef7e f   MSVCRT:ucrt_stubs.obj
 0001:0001df7e       ___acrt_thread_detach      1001ef7e f   MSVCRT:ucrt_stubs.obj
 0001:0001df7e       ___acrt_uninitialize       1001ef7e f   MSVCRT:ucrt_stubs.obj
 0001:0001df7e       ___acrt_uninitialize_critical 1001ef7e f   MSVCRT:ucrt_stubs.obj
 0001:0001df7e       ___scrt_stub_for_acrt_initialize 1001ef7e f   MSVCRT:ucrt_stubs.obj
 0001:0001df7e       ___scrt_stub_for_acrt_thread_attach 1001ef7e f   MSVCRT:ucrt_stubs.obj
 0001:0001df7e       ___scrt_stub_for_acrt_thread_detach 1001ef7e f   MSVCRT:ucrt_stubs.obj
 0001:0001df7e       ___scrt_stub_for_acrt_uninitialize 1001ef7e f   MSVCRT:ucrt_stubs.obj
 0001:0001df7e       ___scrt_stub_for_acrt_uninitialize_critical 1001ef7e f   MSVCRT:ucrt_stubs.obj
 0001:0001df7e       ___vcrt_initialize         1001ef7e f   MSVCRT:ucrt_stubs.obj
 0001:0001df7e       ___vcrt_thread_attach      1001ef7e f   MSVCRT:ucrt_stubs.obj
 0001:0001df7e       ___vcrt_thread_detach      1001ef7e f   MSVCRT:ucrt_stubs.obj
 0001:0001df7e       ___vcrt_uninitialize       1001ef7e f   MSVCRT:ucrt_stubs.obj
 0001:0001df7e       ___vcrt_uninitialize_critical 1001ef7e f   MSVCRT:ucrt_stubs.obj
 0001:0001df81       __filter_x86_sse2_floating_point_exception 1001ef81 f   MSVCRT:x86_exception_filter.obj
 0001:0001df81       __filter_x86_sse2_floating_point_exception_default 1001ef81 f   MSVCRT:x86_exception_filter.obj
 0002:00000000       __imp__QueryPerformanceCounter@4 1001f000     kernel32:KERNEL32.dll
 0002:00000004       __imp__IsDebuggerPresent@0 1001f004     kernel32:KERNEL32.dll
 0002:00000008       __imp__InitializeSListHead@4 1001f008     kernel32:KERNEL32.dll
 0002:0000000c       __imp__IsProcessorFeaturePresent@4 1001f00c     kernel32:KERNEL32.dll
 0002:00000010       __imp__UnhandledExceptionFilter@4 1001f010     kernel32:KERNEL32.dll
 0002:00000014       __imp__SetUnhandledExceptionFilter@4 1001f014     kernel32:KERNEL32.dll
 0002:00000018       __imp__GetCurrentProcess@0 1001f018     kernel32:KERNEL32.dll
 0002:0000001c       __imp__TerminateProcess@8  1001f01c     kernel32:KERNEL32.dll
 0002:00000020       __imp__GetSystemTimeAsFileTime@4 1001f020     kernel32:KERNEL32.dll
 0002:00000024       __imp__GetCurrentProcessId@0 1001f024     kernel32:KERNEL32.dll
 0002:00000028       __imp__GetCurrentThreadId@0 1001f028     kernel32:KERNEL32.dll
 0002:0000002c       __imp__DisableThreadLibraryCalls@4 1001f02c     kernel32:KERNEL32.dll
 0002:00000030       \177KERNEL32_NULL_THUNK_DATA 1001f030     kernel32:KERNEL32.dll
 0002:00000034       __imp____std_type_info_destroy_list 1001f034     vcruntime:VCRUNTIME140.dll
 0002:00000038       __imp___except_handler4_common 1001f038     vcruntime:VCRUNTIME140.dll
 0002:0000003c       __imp__memmove             1001f03c     vcruntime:VCRUNTIME140.dll
 0002:00000040       __imp__longjmp             1001f040     vcruntime:VCRUNTIME140.dll
 0002:00000044       __imp___setjmp3            1001f044     vcruntime:VCRUNTIME140.dll
 0002:00000048       __imp__memcpy              1001f048     vcruntime:VCRUNTIME140.dll
 0002:0000004c       __imp__memset              1001f04c     vcruntime:VCRUNTIME140.dll
 0002:00000050       \177VCRUNTIME140_NULL_THUNK_DATA 1001f050     vcruntime:VCRUNTIME140.dll
 0002:00000054       __imp__getenv              1001f054     ucrt:api-ms-win-crt-environment-l1-1-0.dll
 0002:00000058       \177api-ms-win-crt-environment-l1-1-0_NULL_THUNK_DATA 1001f058     ucrt:api-ms-win-crt-environment-l1-1-0.dll
 0002:0000005c       __imp__calloc              1001f05c     ucrt:api-ms-win-crt-heap-l1-1-0.dll
 0002:00000060       __imp__free                1001f060     ucrt:api-ms-win-crt-heap-l1-1-0.dll
 0002:00000064       __imp__malloc              1001f064     ucrt:api-ms-win-crt-heap-l1-1-0.dll
 0002:00000068       \177api-ms-win-crt-heap-l1-1-0_NULL_THUNK_DATA 1001f068     ucrt:api-ms-win-crt-heap-l1-1-0.dll
 0002:0000006c       __imp___cexit              1001f06c     ucrt:api-ms-win-crt-runtime-l1-1-0.dll
 0002:00000070       __imp___initialize_onexit_table 1001f070     ucrt:api-ms-win-crt-runtime-l1-1-0.dll
 0002:00000074       __imp___execute_onexit_table 1001f074     ucrt:api-ms-win-crt-runtime-l1-1-0.dll
 0002:00000078       __imp___initterm           1001f078     ucrt:api-ms-win-crt-runtime-l1-1-0.dll
 0002:0000007c       __imp___initterm_e         1001f07c     ucrt:api-ms-win-crt-runtime-l1-1-0.dll
 0002:00000080       __imp___seh_filter_dll     1001f080     ucrt:api-ms-win-crt-runtime-l1-1-0.dll
 0002:00000084       __imp___configure_narrow_argv 1001f084     ucrt:api-ms-win-crt-runtime-l1-1-0.dll
 0002:00000088       __imp___initialize_narrow_environment 1001f088     ucrt:api-ms-win-crt-runtime-l1-1-0.dll
 0002:0000008c       \177api-ms-win-crt-runtime-l1-1-0_NULL_THUNK_DATA 1001f08c     ucrt:api-ms-win-crt-runtime-l1-1-0.dll
 0002:00000090       __imp____stdio_common_vfprintf 1001f090     ucrt:api-ms-win-crt-stdio-l1-1-0.dll
 0002:00000094       __imp____acrt_iob_func     1001f094     ucrt:api-ms-win-crt-stdio-l1-1-0.dll
 0002:00000098       __imp____stdio_common_vsscanf 1001f098     ucrt:api-ms-win-crt-stdio-l1-1-0.dll
 0002:0000009c       \177api-ms-win-crt-stdio-l1-1-0_NULL_THUNK_DATA 1001f09c     ucrt:api-ms-win-crt-stdio-l1-1-0.dll
 0002:000000a0       __imp__JNU_GetEnv@8        1001f0a0     java:java.dll
 0002:000000a4       __imp__jio_snprintf        1001f0a4     java:java.dll
 0002:000000a8       __imp__JNU_ThrowNullPointerException@8 1001f0a8     java:java.dll
 0002:000000ac       __imp__JNU_ThrowByName@12  1001f0ac     java:java.dll
 0002:000000b0       \177java_NULL_THUNK_DATA   1001f0b0     java:java.dll
 0002:000000b4       ___guard_check_icall_fptr  1001f0b4     MSVCRT:guard_support.obj
 0002:000000b8       ___castguard_check_failure_os_handled_fptr 1001f0b8     MSVCRT:guard_support.obj
 0002:000000bc       ___xc_a                    1001f0bc     MSVCRT:initializers.obj
 0002:000000c0       ___xc_z                    1001f0c0     MSVCRT:initializers.obj
 0002:000000c4       ___xi_a                    1001f0c4     MSVCRT:initializers.obj
 0002:000000c8       ___xi_z                    1001f0c8     MSVCRT:initializers.obj
 0002:000000cc       ___xp_a                    1001f0cc     MSVCRT:initializers.obj
 0002:000000d0       ___xp_z                    1001f0d0     MSVCRT:initializers.obj
 0002:000000d4       ___xt_a                    1001f0d4     MSVCRT:initializers.obj
 0002:000000d8       ___xt_z                    1001f0d8     MSVCRT:initializers.obj
 0002:000000e0       ??_C@_0BE@LOJEHOGK@Initializing?5Reader@ 1001f0e0     imageioJPEG.obj
 0002:000000f4       ??_C@_0BL@ENCPOIKC@java?1lang?1OutOfMemoryError@ 1001f0f4     imageioJPEG.obj
 0002:00000110       ??_C@_0BF@GNONHPOP@Setting?5Pixel?5Buffer@ 1001f110     imageioJPEG.obj
 0002:00000128       ??_C@_0BL@PAGFHBFL@javax?1imageio?1IIOException@ 1001f128     imageioJPEG.obj
 0002:00000144       ??_C@_0DF@EJNALACK@Invalid?5icc?5profile?3?5inconsiste@ 1001f144     imageioJPEG.obj
 0002:0000017c       ??_C@_0CJ@PKIHEMMA@Invalid?5icc?5profile?3?5bad?5sequen@ 1001f17c     imageioJPEG.obj
 0002:000001a8       ??_C@_0DA@GLMLOKJH@Invalid?5icc?5profile?3?5duplicate?5@ 1001f1a8     imageioJPEG.obj
 0002:000001d8       ??_C@_0DD@PBCIMJPM@Invalid?5icc?5profile?3?5invalid?5nu@ 1001f1d8     imageioJPEG.obj
 0002:0000020c       ??_C@_0CN@PIKPANEC@Invalid?5icc?5profile?3?5missing?5se@ 1001f20c     imageioJPEG.obj
 0002:0000023c       ??_C@_0CJ@HIEMCHIB@Invalid?5icc?5profile?3?5invalid?5da@ 1001f23c     imageioJPEG.obj
 0002:00000268       ??_C@_0CO@ILDJFFGN@Invalid?5icc?5profile?3?5found?5only@ 1001f268     imageioJPEG.obj
 0002:00000298       ??_C@_0BE@JBLDAGLI@Reading?5ICC?5profile@ 1001f298     imageioJPEG.obj
 0002:000002ac       ??_C@_0CF@EJBMEBBP@Unable?5to?5pin?5icc?5profile?5data?5@ 1001f2ac     imageioJPEG.obj
 0002:000002d4       ??_C@_07HGNEOLPD@?$CI?$FLBII?$CJI@ 1001f2d4     imageioJPEG.obj
 0002:000002dc       ??_C@_0O@BACJPOFC@readInputData@ 1001f2dc     imageioJPEG.obj
 0002:000002ec       ??_C@_04BMPAOJO@?$CIJ?$CJJ@ 1001f2ec     imageioJPEG.obj
 0002:000002f4       ??_C@_0P@CHNKCPBH@skipInputBytes@ 1001f2f4     imageioJPEG.obj
 0002:00000304       ??_C@_04PFANPMCN@?$CII?$CJV@ 1001f304     imageioJPEG.obj
 0002:0000030c       ??_C@_0BA@CDPOJDB@warningOccurred@ 1001f30c     imageioJPEG.obj
 0002:0000031c       ??_C@_0BG@IKDDPPGD@?$CILjava?1lang?1String?$DL?$CJV@ 1001f31c     imageioJPEG.obj
 0002:00000334       ??_C@_0BD@EDGGINKI@warningWithMessage@ 1001f334     imageioJPEG.obj
 0002:00000348       ??_C@_0L@NCAMOCKO@?$CIIIIII?$FLB?$CJV@ 1001f348     imageioJPEG.obj
 0002:00000354       ??_C@_0N@MNKCGBOF@setImageData@ 1001f354     imageioJPEG.obj
 0002:00000364       ??_C@_05IPOMILEE@?$CIIZ?$CJV@ 1001f364     imageioJPEG.obj
 0002:0000036c       ??_C@_0N@NGMIGEIH@acceptPixels@ 1001f36c     imageioJPEG.obj
 0002:0000037c       ??_C@_0M@MNIOMPPJ@passStarted@ 1001f37c     imageioJPEG.obj
 0002:00000388       ??_C@_03GAEACAIP@?$CI?$CJV@ 1001f388     imageioJPEG.obj
 0002:0000038c       ??_C@_0N@JHOJIANF@passComplete@ 1001f38c     imageioJPEG.obj
 0002:0000039c       ??_C@_08FJPDKMKL@pushBack@ 1001f39c     imageioJPEG.obj
 0002:000003a8       ??_C@_0O@ENCADKKM@skipPastImage@ 1001f3a8     imageioJPEG.obj
 0002:000003b8       ??_C@_02EBOMBDPA@?$FLI@    1001f3b8     imageioJPEG.obj
 0002:000003bc       ??_C@_06NDKJHNCM@qTable@   1001f3bc     imageioJPEG.obj
 0002:000003c4       ??_C@_02PBMBOJCL@?$FLS@    1001f3c4     imageioJPEG.obj
 0002:000003c8       ??_C@_07HLHALEDB@lengths@  1001f3c8     imageioJPEG.obj
 0002:000003d0       ??_C@_06GEKOPAHD@values@   1001f3d0     imageioJPEG.obj
 0002:000003d8       ??_C@_0CJ@FAHHFKDG@Attempting?5to?5use?5reader?5after?5@ 1001f3d8     imageioJPEG.obj
 0002:00000404       ??_C@_0CA@EJBFMCPI@java?1lang?1IllegalStateException@ 1001f404     imageioJPEG.obj
 0002:00000424       ??_C@_0BB@BBPIIEJP@Array?5pin?5failed@ 1001f424     imageioJPEG.obj
 0002:00000438       ??_C@_0CF@OPBCJGNA@Invalid?5argument?5to?5native?5read@ 1001f438     imageioJPEG.obj
 0002:00000460       ??_C@_0BC@OMEGECOD@Initializing?5Read@ 1001f460     imageioJPEG.obj
 0002:00000474       ??_C@_0CE@LPFBCDGM@Invalid?5number?5of?5output?5compon@ 1001f474     imageioJPEG.obj
 0002:00000498       ??_C@_0BE@KOGPEOLP@Reading?5JPEG?5Stream@ 1001f498     imageioJPEG.obj
 0002:000004ac       ??_C@_0BK@PBGJCCG@Output?5buffer?5not?5pinned?$CB@ 1001f4ac     imageioJPEG.obj
 0002:000004c8       ??_C@_07LLIOOFGN@?$CI?$FLBII?$CJV@ 1001f4c8     imageioJPEG.obj
 0002:000004d0       ??_C@_0BA@MONANPK@writeOutputData@ 1001f4d0     imageioJPEG.obj
 0002:000004e0       ??_C@_0O@BLOPFHGH@writeMetadata@ 1001f4e0     imageioJPEG.obj
 0002:000004f0       ??_C@_0L@EKFGKJEH@grabPixels@ 1001f4f0     imageioJPEG.obj
 0002:000004fc       ??_C@_0BE@JCBGHPLA@Initializing?5Writer@ 1001f4fc     imageioJPEG.obj
 0002:00000510       ??_C@_0CJ@MCECMHCD@Attempting?5to?5use?5writer?5after?5@ 1001f510     imageioJPEG.obj
 0002:0000053c       ??_C@_0CG@JKMPIIDL@Invalid?5argument?5to?5native?5writ@ 1001f53c     imageioJPEG.obj
 0002:00000564       ??_C@_0O@FAOJELCO@Invalid?5Image@ 1001f564     imageioJPEG.obj
 0002:00000574       ??_C@_0BE@NMJJBJJA@Writing?5JPEG?5Stream@ 1001f574     imageioJPEG.obj
 0002:00000588       __real@3ff0000000000000    1001f588     jcapimin.obj
 0002:00000590       __xmm@00000003000000020000000100000000 1001f590     jccolor.obj
 0002:000005a0       __xmm@00001d2f00001d2f00001d2f00001d2f 1001f5a0     jccolor.obj
 0002:000005b0       __xmm@00004c8b00004c8b00004c8b00004c8b 1001f5b0     jccolor.obj
 0002:000005c0       __xmm@00008000000080000000800000008000 1001f5c0     jccolor.obj
 0002:000005d0       __xmm@00009646000096460000964600009646 1001f5d0     jccolor.obj
 0002:000005e0       __xmm@00807fff00807fff00807fff00807fff 1001f5e0     jccolor.obj
 0002:000005f0       __xmm@ffff94d1ffff94d1ffff94d1ffff94d1 1001f5f0     jccolor.obj
 0002:00000600       __xmm@ffffab33ffffab33ffffab33ffffab33 1001f600     jccolor.obj
 0002:00000610       __xmm@ffffd4cdffffd4cdffffd4cdffffd4cd 1001f610     jccolor.obj
 0002:00000620       __xmm@ffffeb2fffffeb2fffffeb2fffffeb2f 1001f620     jccolor.obj
 0002:000006f0       __real@3fd1a855de72ab5d    1001f6f0     jcdctmgr.obj
 0002:000006f8       __real@3fe1517a7bc720bb    1001f6f8     jcdctmgr.obj
 0002:00000700       __real@3fe92469c0a7bf3b    1001f700     jcdctmgr.obj
 0002:00000708       __real@3ff2d062ef6c11aa    1001f708     jcdctmgr.obj
 0002:00000710       __real@3ff4e7ae914d6fca    1001f710     jcdctmgr.obj
 0002:00000718       __real@3ff63150b14861ef    1001f718     jcdctmgr.obj
 0002:00000720       __real@4020000000000000    1001f720     jcdctmgr.obj
 0002:00000728       __real@46800100            1001f728     jcdctmgr.obj
 0002:00000730       __xmm@00000400000004000000040000000400 1001f730     jcdctmgr.obj
 0002:00000740       __xmm@40004000400040004000400040004000 1001f740     jcdctmgr.obj
 0002:00000750       __xmm@46800100468001004680010046800100 1001f750     jcdctmgr.obj
 0002:00000be0       __xmm@00000800000008000000080000000800 1001fbe0     jddctmgr.obj
 0002:00000cf0       _jMsgTable                 1001fcf0     jerror.obj
 0002:00000ee4       ??_C@_0BG@MIBALFBH@Bogus?5message?5code?5?$CFd@ 1001fee4     jerror.obj
 0002:00000efc       ??_C@_0DJ@KONAFFHE@Sorry?0?5there?5are?5legal?5restrict@ 1001fefc     jerror.obj
 0002:00000f38       ??_C@_0CA@FDMPGPNI@ALIGN_TYPE?5is?5wrong?0?5please?5fix@ 1001ff38     jerror.obj
 0002:00000f58       ??_C@_0CF@DENLILGA@MAX_ALLOC_CHUNK?5is?5wrong?0?5pleas@ 1001ff58     jerror.obj
 0002:00000f80       ??_C@_0BK@DKALDNKG@Bogus?5buffer?5control?5mode@ 1001ff80     jerror.obj
 0002:00000f9c       ??_C@_0BP@ONFLCDHG@Invalid?5component?5ID?5?$CFd?5in?5SOS@ 1001ff9c     jerror.obj
 0002:00000fbc       ??_C@_0BN@OJEJKKDL@DCT?5coefficient?5out?5of?5range@ 1001ffbc     jerror.obj
 0002:00000fdc       ??_C@_0CI@MBJANLAP@IDCT?5output?5block?5size?5?$CFd?5not?5s@ 1001ffdc     jerror.obj
 0002:00001004       ??_C@_0BP@EOFJNLFD@Bogus?5Huffman?5table?5definition@ 10020004     jerror.obj
 0002:00001024       ??_C@_0BH@BGDIGLHC@Bogus?5input?5colorspace@ 10020024     jerror.obj
 0002:0000103c       ??_C@_0BG@NEGIHEMC@Bogus?5JPEG?5colorspace@ 1002003c     jerror.obj
 0002:00001054       ??_C@_0BE@OGLAEMOG@Bogus?5marker?5length@ 10020054     jerror.obj
 0002:00001068       ??_C@_0DN@ELFKFKL@Wrong?5JPEG?5library?5version?3?5lib@ 10020068     jerror.obj
 0002:000010a8       ??_C@_0DA@HLEOHNPA@Sampling?5factors?5too?5large?5for?5@ 100200a8     jerror.obj
 0002:000010d8       ??_C@_0BM@OEMICEFD@Invalid?5memory?5pool?5code?5?$CFd@ 100200d8     jerror.obj
 0002:000010f4       ??_C@_0CD@LDBDNLHK@Unsupported?5JPEG?5data?5precision@ 100200f4     jerror.obj
 0002:00001118       ??_C@_0DH@LNGGEGOL@Invalid?5progressive?5parameters?5@ 10020118     jerror.obj
 0002:00001150       ??_C@_0DH@HIKEGPKP@Invalid?5progressive?5parameters?5@ 10020150     jerror.obj
 0002:00001188       ??_C@_0BH@HMMHPOPE@Bogus?5sampling?5factors@ 10020188     jerror.obj
 0002:000011a0       ??_C@_0CA@MJDDICLK@Invalid?5scan?5script?5at?5entry?5?$CFd@ 100201a0     jerror.obj
 0002:000011c0       ??_C@_0CK@BAMFIBMM@Improper?5call?5to?5JPEG?5library?5i@ 100201c0     jerror.obj
 0002:000011f0       ??_C@_0EN@DKAEGIBH@JPEG?5parameter?5struct?5mismatch?3@ 100201f0     jerror.obj
 0002:00001240       ??_C@_0BL@CBOEEPLK@Bogus?5virtual?5array?5access@ 10020240     jerror.obj
 0002:0000125c       ??_C@_0CL@JKHIPJLJ@Buffer?5passed?5to?5JPEG?5library?5i@ 1002025c     jerror.obj
 0002:00001288       ??_C@_0BM@PKHCPJDH@Suspension?5not?5allowed?5here@ 10020288     jerror.obj
 0002:000012a4       ??_C@_0CF@LAEFHNAH@CCIR601?5sampling?5not?5implemente@ 100202a4     jerror.obj
 0002:000012cc       ??_C@_0CG@BEBDNOCG@Too?5many?5color?5components?3?5?$CFd?0?5@ 100202cc     jerror.obj
 0002:000012f4       ??_C@_0CF@JDLOPNGO@Unsupported?5color?5conversion?5re@ 100202f4     jerror.obj
 0002:0000131c       ??_C@_0BD@LDBBBMFL@Bogus?5DAC?5index?5?$CFd@ 1002031c     jerror.obj
 0002:00001330       ??_C@_0BF@CLIOOJFM@Bogus?5DAC?5value?50x?$CFx@ 10020330     jerror.obj
 0002:00001348       ??_C@_0BD@KJHFPHIC@Bogus?5DHT?5index?5?$CFd@ 10020348     jerror.obj
 0002:0000135c       ??_C@_0BD@DIMECAOP@Bogus?5DQT?5index?5?$CFd@ 1002035c     jerror.obj
 0002:00001370       ??_C@_0CF@DAGGEAPM@Empty?5JPEG?5image?5?$CIDNL?5not?5suppo@ 10020370     jerror.obj
 0002:00001398       ??_C@_0BF@CPNENPBA@Read?5from?5EMS?5failed@ 10020398     jerror.obj
 0002:000013b0       ??_C@_0BE@DGJBKIEB@Write?5to?5EMS?5failed@ 100203b0     jerror.obj
 0002:000013c4       ??_C@_0CB@DMGINPNE@Didn?8t?5expect?5more?5than?5one?5sca@ 100203c4     jerror.obj
 0002:000013e8       ??_C@_0BG@BALCKDNL@Input?5file?5read?5error@ 100203e8     jerror.obj
 0002:00001400       ??_C@_0CP@IDOBLGGD@Output?5file?5write?5error?5?9?9?9?5out@ 10020400     jerror.obj
 0002:00001430       ??_C@_0CI@EKDDDHFF@Fractional?5sampling?5not?5impleme@ 10020430     jerror.obj
 0002:00001458       ??_C@_0CB@LLDOGNPJ@Huffman?5code?5size?5table?5overflo@ 10020458     jerror.obj
 0002:0000147c       ??_C@_0CB@LFBMFPHI@Missing?5Huffman?5code?5table?5entr@ 1002047c     jerror.obj
 0002:000014a0       ??_C@_0CP@EKFPGPNP@Maximum?5supported?5image?5dimensi@ 100204a0     jerror.obj
 0002:000014d0       ??_C@_0BB@JJAIKFBB@Empty?5input?5file@ 100204d0     jerror.obj
 0002:000014e4       ??_C@_0BM@KEKMMNGA@Premature?5end?5of?5input?5file@ 100204e4     jerror.obj
 0002:00001500       ??_C@_0DO@OPNPKGO@Cannot?5transcode?5due?5to?5multipl@ 10020500     jerror.obj
 0002:00001540       ??_C@_0CH@NIBDNILP@Scan?5script?5does?5not?5transmit?5a@ 10020540     jerror.obj
 0002:00001568       ??_C@_0CH@EFBBPPCK@Invalid?5color?5quantization?5mode@ 10020568     jerror.obj
 0002:00001590       ??_C@_0BE@EOAAHHJ@Not?5implemented?5yet@ 10020590     jerror.obj
 0002:000015a4       ??_C@_0CO@BEHINNOI@Requested?5feature?5was?5omitted?5a@ 100205a4     jerror.obj
 0002:000015d4       ??_C@_0BM@HJHFKLAF@Backing?5store?5not?5supported@ 100205d4     jerror.obj
 0002:000015f0       ??_C@_0CF@BKANFCCL@Huffman?5table?50x?$CF02x?5was?5not?5de@ 100205f0     jerror.obj
 0002:00001618       ??_C@_0CC@BKPLBDLJ@JPEG?5datastream?5contains?5no?5ima@ 10020618     jerror.obj
 0002:0000163c       ??_C@_0CK@CCHKIENB@Quantization?5table?50x?$CF02x?5was?5n@ 1002063c     jerror.obj
 0002:00001668       ??_C@_0CL@GNLFDFCL@Not?5a?5JPEG?5file?3?5starts?5with?50x@ 10020668     jerror.obj
 0002:00001694       ??_C@_0BO@DJPLELIB@Insufficient?5memory?5?$CIcase?5?$CFd?$CJ@ 10020694     jerror.obj
 0002:000016b4       ??_C@_0CO@HPDBAEEA@Cannot?5quantize?5more?5than?5?$CFd?5co@ 100206b4     jerror.obj
 0002:000016e4       ??_C@_0CI@PLMPLCNO@Cannot?5quantize?5to?5fewer?5than?5?$CF@ 100206e4     jerror.obj
 0002:0000170c       ??_C@_0CH@NHMNHHIB@Cannot?5quantize?5to?5more?5than?5?$CFd@ 1002070c     jerror.obj
 0002:00001734       ??_C@_0CN@IHJJJAFJ@Invalid?5JPEG?5file?5structure?3?5tw@ 10020734     jerror.obj
 0002:00001764       ??_C@_0DA@GJIJGINK@Invalid?5JPEG?5file?5structure?3?5mi@ 10020764     jerror.obj
 0002:00001794       ??_C@_0CK@HMKECJK@Unsupported?5JPEG?5process?3?5SOF?5t@ 10020794     jerror.obj
 0002:000017c0       ??_C@_0CN@HGJCMLNE@Invalid?5JPEG?5file?5structure?3?5tw@ 100207c0     jerror.obj
 0002:000017f0       ??_C@_0CM@HONLBDPH@Invalid?5JPEG?5file?5structure?3?5SO@ 100207f0     jerror.obj
 0002:0000181c       ??_C@_0CD@POKNOPOF@Failed?5to?5create?5temporary?5file@ 1002081c     jerror.obj
 0002:00001840       ??_C@_0BO@EEPJGHHI@Read?5failed?5on?5temporary?5file@ 10020840     jerror.obj
 0002:00001860       ??_C@_0BO@GOBJOAAI@Seek?5failed?5on?5temporary?5file@ 10020860     jerror.obj
 0002:00001880       ??_C@_0DG@KALDLIJB@Write?5failed?5on?5temporary?5file?5@ 10020880     jerror.obj
 0002:000018b8       ??_C@_0CK@EPADOAKC@Application?5transferred?5too?5few@ 100208b8     jerror.obj
 0002:000018e4       ??_C@_0BP@BPKOBOIP@Unsupported?5marker?5type?50x?$CF02x@ 100208e4     jerror.obj
 0002:00001904       ??_C@_0CD@GCLFJCHC@Virtual?5array?5controller?5messed@ 10020904     jerror.obj
 0002:00001928       ??_C@_0CH@LJLHCCHC@Image?5too?5wide?5for?5this?5impleme@ 10020928     jerror.obj
 0002:00001950       ??_C@_0BF@EKLGFGNM@Read?5from?5XMS?5failed@ 10020950     jerror.obj
 0002:00001968       ??_C@_0BE@FDPDCBIN@Write?5to?5XMS?5failed@ 10020968     jerror.obj
 0002:0000197c       ??_C@_0CD@IMBKIDCD@Copyright?5?$CIC?$CJ?51998?0?5Thomas?5G?4?5L@ 1002097c     jerror.obj
 0002:000019a0       ??_C@_0BA@LIJBPGPA@6b?5?527?9Mar?91998@ 100209a0     jerror.obj
 0002:000019b0       ??_C@_0DO@EGLODMBB@Caution?3?5quantization?5tables?5ar@ 100209b0     jerror.obj
 0002:000019f0       ??_C@_0EC@EHPKAOHA@Adobe?5APP14?5marker?3?5version?5?$CFd?0@ 100209f0     jerror.obj
 0002:00001a34       ??_C@_0CK@HCPFFNKJ@Unknown?5APP0?5marker?5?$CInot?5JFIF?$CJ?0@ 10020a34     jerror.obj
 0002:00001a60       ??_C@_0CM@CAEPHFAA@Unknown?5APP14?5marker?5?$CInot?5Adobe@ 10020a60     jerror.obj
 0002:00001a8c       ??_C@_0CH@KIJGKPAA@Define?5Arithmetic?5Table?50x?$CF02x?3@ 10020a8c     jerror.obj
 0002:00001ab4       ??_C@_0BM@MDIEILCE@Define?5Huffman?5Table?50x?$CF02x@ 10020ab4     jerror.obj
 0002:00001ad0       ??_C@_0CL@KLDOJIKN@Define?5Quantization?5Table?5?$CFd?5?5p@ 10020ad0     jerror.obj
 0002:00001afc       ??_C@_0BL@EMFIKBEK@Define?5Restart?5Interval?5?$CFu@ 10020afc     jerror.obj
 0002:00001b18       ??_C@_0BE@IPCOOGDJ@Freed?5EMS?5handle?5?$CFu@ 10020b18     jerror.obj
 0002:00001b2c       ??_C@_0BH@GIPOLIGC@Obtained?5EMS?5handle?5?$CFu@ 10020b2c     jerror.obj
 0002:00001b44       ??_C@_0N@HJHFKELG@End?5Of?5Image@ 10020b44     jerror.obj
 0002:00001b54       ??_C@_0CI@FKGPAJC@?5?5?5?5?5?5?5?5?$CF3d?5?$CF3d?5?$CF3d?5?$CF3d?5?$CF3d?5?$CF3d@ 10020b54     jerror.obj
 0002:00001b7c       ??_C@_0DF@LOKNABIG@JFIF?5APP0?5marker?3?5version?5?$CFd?4?$CF0@ 10020b7c     jerror.obj
 0002:00001bb4       ??_C@_0DM@JLHNPIBE@Warning?3?5thumbnail?5image?5size?5d@ 10020bb4     jerror.obj
 0002:00001bf0       ??_C@_0CO@KKPHGHBA@JFIF?5extension?5marker?3?5type?50x?$CF@ 10020bf0     jerror.obj
 0002:00001c20       ??_C@_0CB@BADBMAAB@?5?5?5?5with?5?$CFd?5x?5?$CFd?5thumbnail?5imag@ 10020c20     jerror.obj
 0002:00001c44       ??_C@_0CH@EHHJCMGA@Miscellaneous?5marker?50x?$CF02x?0?5le@ 10020c44     jerror.obj
 0002:00001c6c       ??_C@_0BJ@COPODLDN@Unexpected?5marker?50x?$CF02x@ 10020c6c     jerror.obj
 0002:00001c88       ??_C@_0CI@GHPOCOCL@?5?5?5?5?5?5?5?5?$CF4u?5?$CF4u?5?$CF4u?5?$CF4u?5?$CF4u?5?$CF4u@ 10020c88     jerror.obj
 0002:00001cb0       ??_C@_0CD@CNNAOOFA@Quantizing?5to?5?$CFd?5?$DN?5?$CFd?$CK?$CFd?$CK?$CFd?5col@ 10020cb0     jerror.obj
 0002:00001cd4       ??_C@_0BI@NEIBNACE@Quantizing?5to?5?$CFd?5colors@ 10020cd4     jerror.obj
 0002:00001cec       ??_C@_0CE@FDPBEAOO@Selected?5?$CFd?5colors?5for?5quantiza@ 10020cec     jerror.obj
 0002:00001d10       ??_C@_0CF@NIMOLBCP@At?5marker?50x?$CF02x?0?5recovery?5acti@ 10020d10     jerror.obj
 0002:00001d38       ??_C@_05LLAPAOG@RST?$CFd@  10020d38     jerror.obj
 0002:00001d40       ??_C@_0DJ@PCBCLFML@Smoothing?5not?5supported?5with?5no@ 10020d40     jerror.obj
 0002:00001d7c       ??_C@_0DK@DMINKOGN@Start?5Of?5Frame?50x?$CF02x?3?5width?$DN?$CFu@ 10020d7c     jerror.obj
 0002:00001db8       ??_C@_0BP@EDCAMHHE@?5?5?5?5Component?5?$CFd?3?5?$CFdhx?$CFdv?5q?$DN?$CFd@ 10020db8     jerror.obj
 0002:00001dd8       ??_C@_0P@JLCHJELA@Start?5of?5Image@ 10020dd8     jerror.obj
 0002:00001de8       ??_C@_0BN@BLOOHNC@Start?5Of?5Scan?3?5?$CFd?5components@ 10020de8     jerror.obj
 0002:00001e08       ??_C@_0BO@CDEKFGLC@?5?5?5?5Component?5?$CFd?3?5dc?$DN?$CFd?5ac?$DN?$CFd@ 10020e08     jerror.obj
 0002:00001e28       ??_C@_0BN@GAMIJLDC@?5?5Ss?$DN?$CFd?0?5Se?$DN?$CFd?0?5Ah?$DN?$CFd?0?5Al?$DN?$CFd@ 10020e28     jerror.obj
 0002:00001e48       ??_C@_0BJ@KDCGAOJB@Closed?5temporary?5file?5?$CFs@ 10020e48     jerror.obj
 0002:00001e64       ??_C@_0BJ@GOCABEP@Opened?5temporary?5file?5?$CFs@ 10020e64     jerror.obj
 0002:00001e80       ??_C@_0EC@ELDEPOJP@JFIF?5extension?5marker?3?5JPEG?9com@ 10020e80     jerror.obj
 0002:00001ec4       ??_C@_0DK@JGAPDCJL@JFIF?5extension?5marker?3?5palette?5@ 10020ec4     jerror.obj
 0002:00001f00       ??_C@_0DG@FCFDGNHE@JFIF?5extension?5marker?3?5RGB?5thum@ 10020f00     jerror.obj
 0002:00001f38       ??_C@_0DE@EEJCDLOO@Unrecognized?5component?5IDs?5?$CFd?5?$CF@ 10020f38     jerror.obj
 0002:00001f6c       ??_C@_0BE@FOGGKKAO@Freed?5XMS?5handle?5?$CFu@ 10020f6c     jerror.obj
 0002:00001f80       ??_C@_0BH@LJLGPEFF@Obtained?5XMS?5handle?5?$CFu@ 10020f80     jerror.obj
 0002:00001f98       ??_C@_0CG@KEGHCDOM@Unknown?5Adobe?5color?5transform?5c@ 10020f98     jerror.obj
 0002:00001fc0       ??_C@_0EC@CBCJOINE@Inconsistent?5progression?5sequen@ 10020fc0     jerror.obj
 0002:00002004       ??_C@_0DM@PCOGCKJB@Corrupt?5JPEG?5data?3?5?$CFu?5extraneou@ 10021004     jerror.obj
 0002:00002040       ??_C@_0DB@PGMEPGHN@Corrupt?5JPEG?5data?3?5premature?5en@ 10021040     jerror.obj
 0002:00002074       ??_C@_0CE@PBLDOPKB@Corrupt?5JPEG?5data?3?5bad?5Huffman?5@ 10021074     jerror.obj
 0002:00002098       ??_C@_0CO@ODCCEDLN@Warning?3?5unknown?5JFIF?5revision?5@ 10021098     jerror.obj
 0002:000020c8       ??_C@_0BL@DPFPFMLM@Premature?5end?5of?5JPEG?5file@ 100210c8     jerror.obj
 0002:000020e4       ??_C@_0DI@NFMBADOH@Corrupt?5JPEG?5data?3?5found?5marker@ 100210e4     jerror.obj
 0002:0000211c       ??_C@_0CL@BAKCGOKJ@Invalid?5SOS?5parameters?5for?5sequ@ 1002111c     jerror.obj
 0002:00002148       ??_C@_0CL@OCGBAKPF@Application?5transferred?5too?5man@ 10021148     jerror.obj
 0002:00002174       ??_C@_03OFAPEBGM@?$CFs?6@  10021174     jerror.obj
 0002:00002178       __real@3ec3ef15            10021178     jfdctflt.obj
 0002:0000217c       __real@3f0a8bd4            1002117c     jfdctflt.obj
 0002:00002180       __real@3f3504f3            10021180     jfdctflt.obj
 0002:00002184       __real@3fa73d75            10021184     jfdctflt.obj
 0002:00002188       __real@3f8a8bd4            10021188     jidctflt.obj
 0002:0000218c       __real@3fb504f3            1002118c     jidctflt.obj
 0002:00002190       __real@3fec835e            10021190     jidctflt.obj
 0002:00002194       __real@40273d75            10021194     jidctflt.obj
 0002:000021a8       ??_C@_07OOOLPGAB@JPEGMEM@  100211a8     jmemmgr.obj
 0002:000021b0       ??_C@_04BMELEEFH@?$CFu?$CFc@ 100211b0     jmemmgr.obj
 0002:000021b8       ??_C@_08MLFAPJAK@?$CIIIZZZ?$CJZ@ 100211b8     jpegdecoder.obj
 0002:000021c4       ??_C@_0P@BDIPJFFC@sendHeaderInfo@ 100211c4     jpegdecoder.obj
 0002:000021d4       ??_C@_06ELGPHLGB@?$CI?$FLBI?$CJZ@ 100211d4     jpegdecoder.obj
 0002:000021dc       ??_C@_0L@IINNECMJ@sendPixels@ 100211dc     jpegdecoder.obj
 0002:000021e8       ??_C@_06DMLPEKHA@?$CI?$FLII?$CJZ@ 100211e8     jpegdecoder.obj
 0002:000021f0       ??_C@_04POLDLDMI@read@     100211f0     jpegdecoder.obj
 0002:000021f8       ??_C@_03KNBKCOBB@?$CI?$CJI@ 100211f8     jpegdecoder.obj
 0002:000021fc       ??_C@_09LAIKOIHJ@available@ 100211fc     jpegdecoder.obj
 0002:00002208       ??_C@_0CD@OMFLCCFG@sun?1awt?1image?1ImageFormatExcept@ 10021208     jpegdecoder.obj
 0002:00002340       _jZAGTable                 10021340     jutils.obj
 0002:00002488       __pDefaultRawDllMain       10021488     MSVCRT:dll_dllmain.obj
 0002:00002488       __pRawDllMain              10021488     MSVCRT:dll_dllmain.obj
 0002:00002490       __load_config_used         10021490     MSVCRT:loadcfg.obj
 0002:000025c0       ___safe_se_handler_table   100215c0     <linker-defined>
 0002:000025c4       ___volatile_metadata       100215c4     <linker-defined>
 0002:00002910       ___rtc_iaa                 10021910     MSVCRT:initsect.obj
 0002:00002914       ___rtc_izz                 10021914     MSVCRT:initsect.obj
 0002:00002918       ___rtc_taa                 10021918     MSVCRT:initsect.obj
 0002:0000291c       ___rtc_tzz                 1002191c     MSVCRT:initsect.obj
 0002:00002fe4       __IMPORT_DESCRIPTOR_java   10021fe4     java:java.dll
 0002:00002ff8       __IMPORT_DESCRIPTOR_KERNEL32 10021ff8     kernel32:KERNEL32.dll
 0002:0000300c       __IMPORT_DESCRIPTOR_VCRUNTIME140 1002200c     vcruntime:VCRUNTIME140.dll
 0002:00003020       __IMPORT_DESCRIPTOR_api-ms-win-crt-heap-l1-1-0 10022020     ucrt:api-ms-win-crt-heap-l1-1-0.dll
 0002:00003034       __IMPORT_DESCRIPTOR_api-ms-win-crt-stdio-l1-1-0 10022034     ucrt:api-ms-win-crt-stdio-l1-1-0.dll
 0002:00003048       __IMPORT_DESCRIPTOR_api-ms-win-crt-environment-l1-1-0 10022048     ucrt:api-ms-win-crt-environment-l1-1-0.dll
 0002:0000305c       __IMPORT_DESCRIPTOR_api-ms-win-crt-runtime-l1-1-0 1002205c     ucrt:api-ms-win-crt-runtime-l1-1-0.dll
 0002:00003070       __NULL_IMPORT_DESCRIPTOR   10022070     java:java.dll
 0003:00000000       ___security_cookie_complement 10023000     MSVCRT:gs_cookie.obj
 0003:00000004       ___security_cookie         10023004     MSVCRT:gs_cookie.obj
 0003:00000008       __fltused                  10023008     MSVCRT:fltused.obj
 0003:0000000c       ___isa_enabled             1002300c     MSVCRT:cpu_disp.obj
 0003:00000010       ___scrt_native_dllmain_reason 10023010     MSVCRT:utility.obj
 0003:00000020       ___scrt_ucrt_dll_is_in_use 10023020     MSVCRT:ucrt_stubs.obj
 0003:00000084       ___isa_available           10023084     MSVCRT:cpu_disp.obj
 0003:00000088       ___favor                   10023088     MSVCRT:cpu_disp.obj
 0003:000003b0       ?__type_info_root_node@@3U__type_info_node@@A 100233b0     MSVCRT:tncleanup.obj
 0003:000003b8       ___scrt_current_native_startup_state 100233b8     MSVCRT:utility.obj
 0003:000003bc       ___scrt_native_startup_lock 100233bc     MSVCRT:utility.obj
 0003:000003dc       ___scrt_debugger_hook_flag 100233dc     MSVCRT:utility_desktop.obj
 0003:000003e0       _jvm                       100233e0     <common>
 0003:000003e8       ?_OptionsStorage@?1??__local_stdio_scanf_options@@9@9 100233e8     <common>
 0003:000003f0       ?_OptionsStorage@?1??__local_stdio_printf_options@@9@9 100233f0     <common>
 0003:000003f8       ___dyn_tls_init_callback   100233f8     <common>

 entry point at        0001:0001d92a

 Static symbols

 0000:fffda000       .debug$S                   10000000     jpeg.exp
 0000:fffda000       .debug$S                   10000000     vcruntime:VCRUNTIME140.dll
 0000:fffda000       .debug$S                   10000000     vcruntime:VCRUNTIME140.dll
 0000:fffda000       .debug$S                   10000000     vcruntime:VCRUNTIME140.dll
 0000:fffda000       .debug$S                   10000000     vcruntime:VCRUNTIME140.dll
 0000:fffda000       .debug$S                   10000000     vcruntime:VCRUNTIME140.dll
 0000:fffda000       .debug$S                   10000000     vcruntime:VCRUNTIME140.dll
 0000:fffda000       .debug$S                   10000000     vcruntime:VCRUNTIME140.dll
 0000:fffda000       .debug$S                   10000000     vcruntime:VCRUNTIME140.dll
 0000:fffda000       .debug$S                   10000000     vcruntime:VCRUNTIME140.dll
 0000:fffda000       .debug$S                   10000000     ucrt:api-ms-win-crt-environment-l1-1-0.dll
 0000:fffda000       .debug$S                   10000000     ucrt:api-ms-win-crt-heap-l1-1-0.dll
 0000:fffda000       .debug$S                   10000000     ucrt:api-ms-win-crt-heap-l1-1-0.dll
 0000:fffda000       .debug$S                   10000000     ucrt:api-ms-win-crt-heap-l1-1-0.dll
 0000:fffda000       .debug$S                   10000000     ucrt:api-ms-win-crt-runtime-l1-1-0.dll
 0000:fffda000       .debug$S                   10000000     ucrt:api-ms-win-crt-runtime-l1-1-0.dll
 0000:fffda000       .debug$S                   10000000     ucrt:api-ms-win-crt-runtime-l1-1-0.dll
 0000:fffda000       .debug$S                   10000000     ucrt:api-ms-win-crt-runtime-l1-1-0.dll
 0000:fffda000       .debug$S                   10000000     ucrt:api-ms-win-crt-runtime-l1-1-0.dll
 0000:fffda000       .debug$S                   10000000     ucrt:api-ms-win-crt-runtime-l1-1-0.dll
 0000:fffda000       .debug$S                   10000000     ucrt:api-ms-win-crt-runtime-l1-1-0.dll
 0000:fffda000       .debug$S                   10000000     ucrt:api-ms-win-crt-runtime-l1-1-0.dll
 0000:fffda000       .debug$S                   10000000     ucrt:api-ms-win-crt-runtime-l1-1-0.dll
 0000:fffda000       .debug$S                   10000000     ucrt:api-ms-win-crt-runtime-l1-1-0.dll
 0000:fffda000       .debug$S                   10000000     ucrt:api-ms-win-crt-runtime-l1-1-0.dll
 0000:fffda000       .debug$S                   10000000     ucrt:api-ms-win-crt-runtime-l1-1-0.dll
 0000:fffda000       .debug$S                   10000000     ucrt:api-ms-win-crt-stdio-l1-1-0.dll
 0000:fffda000       .debug$S                   10000000     ucrt:api-ms-win-crt-stdio-l1-1-0.dll
 0000:fffda000       .debug$S                   10000000     ucrt:api-ms-win-crt-stdio-l1-1-0.dll
 0000:fffda000       .debug$S                   10000000     kernel32:KERNEL32.dll
 0000:fffda000       .debug$S                   10000000     kernel32:KERNEL32.dll
 0000:fffda000       .debug$S                   10000000     kernel32:KERNEL32.dll
 0000:fffda000       .debug$S                   10000000     kernel32:KERNEL32.dll
 0000:fffda000       .debug$S                   10000000     kernel32:KERNEL32.dll
 0000:fffda000       .debug$S                   10000000     kernel32:KERNEL32.dll
 0000:fffda000       .debug$S                   10000000     kernel32:KERNEL32.dll
 0000:fffda000       .debug$S                   10000000     kernel32:KERNEL32.dll
 0000:fffda000       .debug$S                   10000000     kernel32:KERNEL32.dll
 0000:fffda000       .debug$S                   10000000     kernel32:KERNEL32.dll
 0000:fffda000       .debug$S                   10000000     kernel32:KERNEL32.dll
 0000:fffda000       .debug$S                   10000000     kernel32:KERNEL32.dll
 0000:fffda000       .debug$S                   10000000     kernel32:KERNEL32.dll
 0000:fffda000       .debug$S                   10000000     kernel32:KERNEL32.dll
 0000:fffda000       .debug$S                   10000000     java:java.dll
 0000:fffda000       .debug$S                   10000000     java:java.dll
 0000:fffda000       .debug$S                   10000000     java:java.dll
 0000:fffda000       .debug$S                   10000000     java:java.dll
 0001:00000000       _GET_ARRAYS                10001000 f   imageioJPEG.obj
 0001:00002b90       _RELEASE_ARRAYS            10003b90 f   imageioJPEG.obj
 0001:00002bf0       _destroyImageioData        10003bf0 f   imageioJPEG.obj
 0001:00002c80       _freeArray                 10003c80 f   imageioJPEG.obj
 0001:00002cc0       _imageio_dispose           10003cc0 f   imageioJPEG.obj
 0001:00002d00       _imageio_empty_output_buffer 10003d00 f   imageioJPEG.obj
 0001:00003110       _imageio_init_destination  10004110 f   imageioJPEG.obj
 0001:00003170       _imageio_reset             10004170 f   imageioJPEG.obj
 0001:00003260       _imageio_set_stream        10004260 f   imageioJPEG.obj
 0001:000034c0       _imageio_term_destination  100044c0 f   imageioJPEG.obj
 0001:000037c0       _initImageioData           100047c0 f   imageioJPEG.obj
 0001:00003ae0       _resetStreamBuffer         10004ae0 f   imageioJPEG.obj
 0001:00003b40       _setHTables                10004b40 f   imageioJPEG.obj
 0001:00003cc0       _setHuffTable              10004cc0 f   imageioJPEG.obj
 0001:00003db0       _setPixelBuffer            10004db0 f   imageioJPEG.obj
 0001:00003e00       _setQTables                10004e00 f   imageioJPEG.obj
 0001:00003f10       _sun_jpeg_error_exit       10004f10 f   imageioJPEG.obj
 0001:00003f10       _sun_jpeg_error_exit       10004f10 f   jpegdecoder.obj
 0001:00003f30       _sun_jpeg_output_message   10004f30 f   imageioJPEG.obj
 0001:00004520       _compress_data             10005520 f   jccoefct.obj
 0001:000047b0       _compress_first_pass       100057b0 f   jccoefct.obj
 0001:000049d0       _compress_output           100059d0 f   jccoefct.obj
 0001:00004d10       _start_iMCU_row            10005d10 f   jccoefct.obj
 0001:00004d80       _start_pass_coef           10005d80 f   jccoefct.obj
 0001:00004e30       _cmyk_ycck_convert         10005e30 f   jccolor.obj
 0001:00004f90       _grayscale_convert         10005f90 f   jccolor.obj
 0001:000051fc       $LN50                      100061fc     jccolor.obj
 0001:00005210       $LN51                      10006210     jccolor.obj
 0001:00005230       _null_convert              10006230 f   jccolor.obj
 0001:000052c0       _null_method               100062c0 f   jccolor.obj
 0001:000052c0       _start_pass_downsample     100062c0 f   jcsample.obj
 0001:000052c0       _start_pass_dcolor         100062c0 f   jdcolor.obj
 0001:000052c0       _finish_pass_1_quant       100062c0 f   jquant1.obj
 0001:000052c0       _finish_pass2              100062c0 f   jquant2.obj
 0001:000052d0       _rgb_gray_convert          100062d0 f   jccolor.obj
 0001:00005380       _rgb_ycc_convert           10006380 f   jccolor.obj
 0001:000054b0       _rgb_ycc_start             100064b0 f   jccolor.obj
 0001:000056a0       _forward_DCT               100066a0 f   jcdctmgr.obj
 0001:00005af0       _forward_DCT_float         10006af0 f   jcdctmgr.obj
 0001:00006350       _start_pass_fdctmgr        10007350 f   jcdctmgr.obj
 0001:000067b0       _emit_bits                 100077b0 f   jchuff.obj
 0001:000068b0       _encode_mcu_gather         100078b0 f   jchuff.obj
 0001:00006a80       _encode_mcu_huff           10007a80 f   jchuff.obj
 0001:00006c90       _encode_one_block          10007c90 f   jchuff.obj
 0001:00006e60       _finish_pass_gather        10007e60 f   jchuff.obj
 0001:00007170       _finish_pass_huff          10008170 f   jchuff.obj
 0001:00007730       _start_pass_huff           10008730 f   jchuff.obj
 0001:00007a10       _process_data_simple_main  10008a10 f   jcmainct.obj
 0001:00007ac0       _start_pass_main           10008ac0 f   jcmainct.obj
 0001:00007b10       _emit_2bytes               10008b10 f   jcmarker.obj
 0001:00007b80       _emit_adobe_app14          10008b80 f   jcmarker.obj
 0001:00007d00       _emit_dht                  10008d00 f   jcmarker.obj
 0001:00007e90       _emit_dqt                  10008e90 f   jcmarker.obj
 0001:00008050       _emit_jfif_app0            10009050 f   jcmarker.obj
 0001:00008280       _emit_marker               10009280 f   jcmarker.obj
 0001:000082f0       _emit_sof                  100092f0 f   jcmarker.obj
 0001:00008480       _emit_sos                  10009480 f   jcmarker.obj
 0001:000086b0       _write_file_header         100096b0 f   jcmarker.obj
 0001:00008700       _write_file_trailer        10009700 f   jcmarker.obj
 0001:00008720       _write_frame_header        10009720 f   jcmarker.obj
 0001:00008820       _write_marker_byte         10009820 f   jcmarker.obj
 0001:00008860       _write_marker_header       10009860 f   jcmarker.obj
 0001:000088a0       _write_scan_header         100098a0 f   jcmarker.obj
 0001:00008980       _write_tables_only         10009980 f   jcmarker.obj
 0001:00008a80       _finish_pass_master        10009a80 f   jcmaster.obj
 0001:00008af0       _initial_setup             10009af0 f   jcmaster.obj
 0001:00008d90       _pass_startup              10009d90 f   jcmaster.obj
 0001:00008dc0       _per_scan_setup            10009dc0 f   jcmaster.obj
 0001:00008fb0       _prepare_for_pass          10009fb0 f   jcmaster.obj
 0001:00009170       _select_scan_parameters    1000a170 f   jcmaster.obj
 0001:00009270       _validate_script           1000a270 f   jcmaster.obj
 0001:00009790       _add_huff_table            1000a790 f   jcparam.obj
 0001:00009870       _fill_dc_scans             1000a870 f   jcparam.obj
 0001:000098e0       _fill_scans                1000a8e0 f   jcparam.obj
 0001:00009dac       $LN23                      1000adac     jcparam.obj
 0001:00009f94       $LN36                      1000af94     jcparam.obj
 0001:0000a250       _emit_bits                 1000b250 f   jcphuff.obj
 0001:0000a3a0       _emit_buffered_bits        1000b3a0 f   jcphuff.obj
 0001:0000a4e0       _emit_eobrun               1000b4e0 f   jcphuff.obj
 0001:0000a590       _emit_restart              1000b590 f   jcphuff.obj
 0001:0000a6a0       _encode_mcu_AC_first       1000b6a0 f   jcphuff.obj
 0001:0000a890       _encode_mcu_AC_refine      1000b890 f   jcphuff.obj
 0001:0000ab20       _encode_mcu_DC_first       1000bb20 f   jcphuff.obj
 0001:0000aca0       _encode_mcu_DC_refine      1000bca0 f   jcphuff.obj
 0001:0000ad60       _finish_pass_gather_phuff  1000bd60 f   jcphuff.obj
 0001:0000ae40       _finish_pass_phuff         1000be40 f   jcphuff.obj
 0001:0000af10       _start_pass_phuff          1000bf10 f   jcphuff.obj
 0001:0000b2a0       _pre_process_context       1000c2a0 f   jcprepct.obj
 0001:0000b4a0       _pre_process_data          1000c4a0 f   jcprepct.obj
 0001:0000b6a0       _start_pass_prep           1000c6a0 f   jcprepct.obj
 0001:0000b6f0       _expand_right_edge         1000c6f0 f   jcsample.obj
 0001:0000b740       _fullsize_downsample       1000c740 f   jcsample.obj
 0001:0000b790       _fullsize_smooth_downsample 1000c790 f   jcsample.obj
 0001:0000b900       _h2v1_downsample           1000c900 f   jcsample.obj
 0001:0000b9a0       _h2v2_downsample           1000c9a0 f   jcsample.obj
 0001:0000ba60       _h2v2_smooth_downsample    1000ca60 f   jcsample.obj
 0001:0000bd10       _int_downsample            1000cd10 f   jcsample.obj
 0001:0000c090       _sep_downsample            1000d090 f   jcsample.obj
 0001:0000c110       _default_decompress_parms  1000d110 f   jdapimin.obj
 0001:0000c390       $LN18                      1000d390     jdapimin.obj
 0001:0000c3a4       $LN17                      1000d3a4     jdapimin.obj
 0001:0000c758       $LN27                      1000d758     jdapimin.obj
 0001:0000c76c       $LN26                      1000d76c     jdapimin.obj
 0001:0000ca20       _output_pass_setup         1000da20 f   jdapistd.obj
 0001:0000cb00       _consume_data              1000db00 f   jdcoefct.obj
 0001:0000cd70       _decompress_data           1000dd70 f   jdcoefct.obj
 0001:0000cf20       _decompress_onepass        1000df20 f   jdcoefct.obj
 0001:0000d1a0       _decompress_smooth_data    1000e1a0 f   jdcoefct.obj
 0001:0000d800       _dummy_consume_data        1000e800 f   jdcoefct.obj
 0001:0000d970       _start_iMCU_row            1000e970 f   jdcoefct.obj
 0001:0000d9e0       _start_input_pass          1000e9e0 f   jdcoefct.obj
 0001:0000da00       _start_output_pass         1000ea00 f   jdcoefct.obj
 0001:0000dba0       _build_ycc_rgb_table       1000eba0 f   jdcolor.obj
 0001:0000dc80       _gray_rgb_convert          1000ec80 f   jdcolor.obj
 0001:0000dcf0       _grayscale_convert         1000ecf0 f   jdcolor.obj
 0001:0000dec4       $LN45                      1000eec4     jdcolor.obj
 0001:0000dee0       _null_convert              1000eee0 f   jdcolor.obj
 0001:0000df70       _ycc_rgb_convert           1000ef70 f   jdcolor.obj
 0001:0000e0b0       _ycck_cmyk_convert         1000f0b0 f   jdcolor.obj
 0001:0000e290       _start_pass                1000f290 f   jddctmgr.obj
 0001:0000e74c       $LN92                      1000f74c     jddctmgr.obj
 0001:0000e770       _decode_mcu                1000f770 f   jdhuff.obj
 0001:0000f150       _start_pass_huff_decoder   10010150 f   jdhuff.obj
 0001:0000f290       _consume_markers           10010290 f   jdinput.obj
 0001:0000f360       _finish_input_pass         10010360 f   jdinput.obj
 0001:0000f380       _initial_setup             10010380 f   jdinput.obj
 0001:0000f5d0       _per_scan_setup            100105d0 f   jdinput.obj
 0001:0000f780       _reset_input_controller    10010780 f   jdinput.obj
 0001:0000f7d0       _start_input_pass          100107d0 f   jdinput.obj
 0001:0000fa30       _process_data_context_main 10010a30 f   jdmainct.obj
 0001:0000fce0       _process_data_crank_post   10010ce0 f   jdmainct.obj
 0001:0000fd10       _process_data_simple_main  10010d10 f   jdmainct.obj
 0001:0000fd90       _start_pass_main           10010d90 f   jdmainct.obj
 0001:0000ff60       _examine_app0              10010f60 f   jdmarker.obj
 0001:000101d0       _examine_app14             100111d0 f   jdmarker.obj
 0001:000102b0       _get_dht                   100112b0 f   jdmarker.obj
 0001:000105c0       _get_dqt                   100115c0 f   jdmarker.obj
 0001:00010880       _get_interesting_appn      10011880 f   jdmarker.obj
 0001:00010a10       _get_sof                   10011a10 f   jdmarker.obj
 0001:00010d60       _get_sos                   10011d60 f   jdmarker.obj
 0001:00011360       _next_marker               10012360 f   jdmarker.obj
 0001:00011460       _read_markers              10012460 f   jdmarker.obj
 0001:00011830       $LN149                     10012830     jdmarker.obj
 0001:00011870       $LN148                     10012870     jdmarker.obj
 0001:00011970       _read_restart_marker       10012970 f   jdmarker.obj
 0001:00011a00       _reset_marker_reader       10012a00 f   jdmarker.obj
 0001:00011a50       _save_marker               10012a50 f   jdmarker.obj
 0001:00011cd0       _skip_variable             10012cd0 f   jdmarker.obj
 0001:00011d90       _finish_output_pass        10012d90 f   jdmaster.obj
 0001:00012040       $LN54                      10013040     jdmaster.obj
 0001:000120a0       _master_selection          100130a0 f   jdmaster.obj
 0001:000123b0       _prepare_for_output_pass   100133b0 f   jdmaster.obj
 0001:00012510       _use_merged_upsample       10013510 f   jdmaster.obj
 0001:00012590       _h2v1_merged_upsample      10013590 f   jdmerge.obj
 0001:00012700       _h2v2_merged_upsample      10013700 f   jdmerge.obj
 0001:00012a50       _merged_1v_upsample        10013a50 f   jdmerge.obj
 0001:00012a90       _merged_2v_upsample        10013a90 f   jdmerge.obj
 0001:00012b50       _start_pass_merged_upsample 10013b50 f   jdmerge.obj
 0001:00012b70       _decode_mcu_AC_first       10013b70 f   jdphuff.obj
 0001:00012db0       _decode_mcu_AC_refine      10013db0 f   jdphuff.obj
 0001:000131a0       _decode_mcu_DC_first       100141a0 f   jdphuff.obj
 0001:000133d0       _decode_mcu_DC_refine      100143d0 f   jdphuff.obj
 0001:00013550       _process_restart           10014550 f   jdphuff.obj
 0001:000135e0       _start_pass_phuff_decoder  100145e0 f   jdphuff.obj
 0001:00013900       _post_process_1pass        10014900 f   jdpostct.obj
 0001:00013980       _post_process_2pass        10014980 f   jdpostct.obj
 0001:00013a20       _post_process_prepass      10014a20 f   jdpostct.obj
 0001:00013ae0       _start_pass_dpost          10014ae0 f   jdpostct.obj
 0001:00013be0       _fullsize_upsample         10014be0 f   jdsample.obj
 0001:00013bf0       _h2v1_fancy_upsample       10014bf0 f   jdsample.obj
 0001:00013cc0       _h2v1_upsample             10014cc0 f   jdsample.obj
 0001:00013d20       _h2v2_fancy_upsample       10014d20 f   jdsample.obj
 0001:00013e70       _h2v2_upsample             10014e70 f   jdsample.obj
 0001:00013ee0       _int_upsample              10014ee0 f   jdsample.obj
 0001:000141c0       _noop_upsample             100151c0 f   jdsample.obj
 0001:000141d0       _sep_upsample              100151d0 f   jdsample.obj
 0001:000142b0       _start_pass_upsample       100152b0 f   jdsample.obj
 0001:000142e0       _emit_message              100152e0 f   jerror.obj
 0001:00014320       _error_exit                10015320 f   jerror.obj
 0001:00014340       _format_message            10015340 f   jerror.obj
 0001:00014490       _output_message            10015490 f   jerror.obj
 0001:00014490       _sun_jpeg_output_message   10015490 f   jpegdecoder.obj
 0001:000144f0       _reset_error_mgr           100154f0 f   jerror.obj
 0001:00019320       _access_virt_barray        1001a320 f   jmemmgr.obj
 0001:00019470       _access_virt_sarray        1001a470 f   jmemmgr.obj
 0001:000195c0       _alloc_barray              1001a5c0 f   jmemmgr.obj
 0001:00019690       _alloc_large               1001a690 f   jmemmgr.obj
 0001:00019760       _alloc_sarray              1001a760 f   jmemmgr.obj
 0001:00019830       _alloc_small               1001a830 f   jmemmgr.obj
 0001:00019970       _do_barray_io              1001a970 f   jmemmgr.obj
 0001:00019a00       _do_sarray_io              1001aa00 f   jmemmgr.obj
 0001:00019a80       _free_pool                 1001aa80 f   jmemmgr.obj
 0001:00019cd0       _realize_virt_arrays       1001acd0 f   jmemmgr.obj
 0001:00019e80       _request_virt_barray       1001ae80 f   jmemmgr.obj
 0001:00019f00       _request_virt_sarray       1001af00 f   jmemmgr.obj
 0001:00019f80       _self_destruct             1001af80 f   jmemmgr.obj
 0001:0001a130       _GET_ARRAYS                1001b130 f   jpegdecoder.obj
 0001:0001aab0       _RELEASE_ARRAYS            1001bab0 f   jpegdecoder.obj
 0001:0001aee0       _alloc_fs_workspace        1001bee0 f   jquant1.obj
 0001:0001af30       _color_quantize            1001bf30 f   jquant1.obj
 0001:0001afe0       _color_quantize3           1001bfe0 f   jquant1.obj
 0001:0001b090       _create_colorindex         1001c090 f   jquant1.obj
 0001:0001b1d0       _create_colormap           1001c1d0 f   jquant1.obj
 0001:0001b4d0       _new_color_map_1_quant     1001c4d0 f   jquant1.obj
 0001:0001b4f0       _quantize3_ord_dither      1001c4f0 f   jquant1.obj
 0001:0001b610       _quantize_fs_dither        1001c610 f   jquant1.obj
 0001:0001b7c0       _quantize_ord_dither       1001c7c0 f   jquant1.obj
 0001:0001b8d0       _start_pass_1_quant        1001c8d0 f   jquant1.obj
 0001:0001ba80       _fill_inverse_cmap         1001ca80 f   jquant2.obj
 0001:0001bcf0       _find_nearby_colors        1001ccf0 f   jquant2.obj
 0001:0001bf00       _finish_pass1              1001cf00 f   jquant2.obj
 0001:0001bf30       _init_error_limit          1001cf30 f   jquant2.obj
 0001:0001c100       _median_cut                1001d100 f   jquant2.obj
 0001:0001c270       _new_color_map_2_quant     1001d270 f   jquant2.obj
 0001:0001c290       _pass2_fs_dither           1001d290 f   jquant2.obj
 0001:0001c570       _pass2_no_dither           1001d570 f   jquant2.obj
 0001:0001c8f0       _prescan_quantize          1001d8f0 f   jquant2.obj
 0001:0001c980       _select_colors             1001d980 f   jquant2.obj
 0001:0001cbc0       _start_pass_2_quant        1001dbc0 f   jquant2.obj
 0001:0001ccf0       _update_box                1001dcf0 f   jquant2.obj
 0001:0001d5ea       ?dllmain_crt_dispatch@@YGHQAUHINSTANCE__@@KQAX@Z 1001e5ea f   MSVCRT:dll_dllmain.obj
 0001:0001d63d       ?dllmain_crt_process_attach@@YAHQAUHINSTANCE__@@QAX@Z 1001e63d f   MSVCRT:dll_dllmain.obj
 0001:0001d744       ?dllmain_crt_process_detach@@YAH_N@Z 1001e744 f   MSVCRT:dll_dllmain.obj
 0001:0001d7f4       ?dllmain_dispatch@@YAHQAUHINSTANCE__@@KQAX@Z 1001e7f4 f   MSVCRT:dll_dllmain.obj
 0001:0001d8ff       ?dllmain_raw@@YGHQAUHINSTANCE__@@KQAX@Z 1001e8ff f   MSVCRT:dll_dllmain.obj
 0001:0001d94d       ___get_entropy             1001e94d f   MSVCRT:gs_support.obj
 0001:0001da3c       ?find_pe_section@@YAPAU_IMAGE_SECTION_HEADER@@QAEI@Z 1001ea3c f   MSVCRT:utility.obj
 0001:0001dea0       $$000000                   1001eea0     MSVCRT:sehprolg4.obj
 0002:00000630       ?aanscales@?8??start_pass_fdctmgr@@9@9 1001f630     jcdctmgr.obj
 0002:000006b0       ?aanscalefactor@?N@??start_pass_fdctmgr@@9@9 1001f6b0     jcdctmgr.obj
 0002:00000760       ?std_luminance_quant_tbl@?1??jSetLQuality@@9@9 1001f760     jcparam.obj
 0002:00000860       ?std_chrominance_quant_tbl@?1??jSetLQuality@@9@9 1001f860     jcparam.obj
 0002:00000960       ?bits_dc_luminance@?1??std_huff_tables@@9@9 1001f960     jcparam.obj
 0002:00000974       ?val_dc_luminance@?1??std_huff_tables@@9@9 1001f974     jcparam.obj
 0002:00000980       ?bits_dc_chrominance@?1??std_huff_tables@@9@9 1001f980     jcparam.obj
 0002:00000994       ?val_dc_chrominance@?1??std_huff_tables@@9@9 1001f994     jcparam.obj
 0002:000009a0       ?bits_ac_luminance@?1??std_huff_tables@@9@9 1001f9a0     jcparam.obj
 0002:000009b8       ?val_ac_luminance@?1??std_huff_tables@@9@9 1001f9b8     jcparam.obj
 0002:00000a5c       ?bits_ac_chrominance@?1??std_huff_tables@@9@9 1001fa5c     jcparam.obj
 0002:00000a70       ?val_ac_chrominance@?1??std_huff_tables@@9@9 1001fa70     jcparam.obj
 0002:00000b18       ?aanscales@?L@??start_pass@@9@9 1001fb18     jddctmgr.obj
 0002:00000b98       ?aanscalefactor@?O@??start_pass@@9@9 1001fb98     jddctmgr.obj
 0002:00000bf0       _extend_test               1001fbf0     jdhuff.obj
 0002:00000c30       _extend_offset             1001fc30     jdhuff.obj
 0002:00000c70       _extend_test               1001fc70     jdphuff.obj
 0002:00000cb0       _extend_offset             1001fcb0     jdphuff.obj
 0002:00002198       _first_pool_slop           10021198     jmemmgr.obj
 0002:000021a0       _extra_pool_slop           100211a0     jmemmgr.obj
 0002:00002230       _base_dither_matrix        10021230     jquant1.obj
 0002:00002330       ?RGB_order@?1??select_ncolors@@9@9 10021330     jquant1.obj
 0002:00002480       _GS_ExceptionPointers      10021480     MSVCRT:gs_report.obj
 0002:00002920       __sehtable$?dllmain_crt_process_attach@@YAHQAUHINSTANCE__@@QAX@Z 10021920     MSVCRT:dll_dllmain.obj
 0002:00002940       __sehtable$?dllmain_crt_process_detach@@YAH_N@Z 10021940     MSVCRT:dll_dllmain.obj
 0002:00002968       __sehtable$?dllmain_dispatch@@YAHQAUHINSTANCE__@@KQAX@Z 10021968     MSVCRT:dll_dllmain.obj
 0002:00002988       __sehtable$___scrt_is_nonwritable_in_current_image 10021988     MSVCRT:utility.obj
 0002:000029b0       .edata                     100219b0     jpeg.exp
 0002:000029d8       rgpv                       100219d8     jpeg.exp
 0002:00002a2c       rgszName                   10021a2c     jpeg.exp
 0002:00002a80       rgwOrd                     10021a80     jpeg.exp
 0002:00002aaa       szName                     10021aaa     jpeg.exp
 0002:00002ab3       $N00001                    10021ab3     jpeg.exp
 0002:00002ac1       $N00002                    10021ac1     jpeg.exp
 0002:00002b01       $N00003                    10021b01     jpeg.exp
 0002:00002b45       $N00004                    10021b45     jpeg.exp
 0002:00002b8e       $N00005                    10021b8e     jpeg.exp
 0002:00002bd2       $N00006                    10021bd2     jpeg.exp
 0002:00002c12       $N00007                    10021c12     jpeg.exp
 0002:00002c58       $N00008                    10021c58     jpeg.exp
 0002:00002ca0       $N00009                    10021ca0     jpeg.exp
 0002:00002ce2       $N00010                    10021ce2     jpeg.exp
 0002:00002d29       $N00011                    10021d29     jpeg.exp
 0002:00002d69       $N00012                    10021d69     jpeg.exp
 0002:00002daa       $N00013                    10021daa     jpeg.exp
 0002:00002dee       $N00014                    10021dee     jpeg.exp
 0002:00002e37       $N00015                    10021e37     jpeg.exp
 0002:00002e7b       $N00016                    10021e7b     jpeg.exp
 0002:00002ebd       $N00017                    10021ebd     jpeg.exp
 0002:00002efb       $N00018                    10021efb     jpeg.exp
 0002:00002f3d       $N00019                    10021f3d     jpeg.exp
 0002:00002f7f       $N00020                    10021f7f     jpeg.exp
 0002:00002faf       $N00021                    10021faf     jpeg.exp
 0002:00003192       .idata$6                   10022192     java:java.dll
 0002:000032c0       .idata$6                   100222c0     kernel32:KERNEL32.dll
 0002:0000333c       .idata$6                   1002233c     vcruntime:VCRUNTIME140.dll
 0002:00003460       .idata$6                   10022460     ucrt:api-ms-win-crt-heap-l1-1-0.dll
 0002:00003480       .idata$6                   10022480     ucrt:api-ms-win-crt-stdio-l1-1-0.dll
 0002:000034a0       .idata$6                   100224a0     ucrt:api-ms-win-crt-environment-l1-1-0.dll
 0002:000034c6       .idata$6                   100224c6     ucrt:api-ms-win-crt-runtime-l1-1-0.dll
 0003:00000028       _JPEGImageReader_readInputDataID 10023028     imageioJPEG.obj
 0003:0000002c       _JPEGImageReader_skipInputBytesID 1002302c     imageioJPEG.obj
 0003:00000030       _JPEGImageReader_warningOccurredID 10023030     imageioJPEG.obj
 0003:00000034       _JPEGImageReader_warningWithMessageID 10023034     imageioJPEG.obj
 0003:00000038       _JPEGImageReader_setImageDataID 10023038     imageioJPEG.obj
 0003:0000003c       _JPEGImageReader_acceptPixelsID 1002303c     imageioJPEG.obj
 0003:00000040       _JPEGImageReader_pushBackID 10023040     imageioJPEG.obj
 0003:00000044       _JPEGImageReader_passStartedID 10023044     imageioJPEG.obj
 0003:00000048       _JPEGImageReader_passCompleteID 10023048     imageioJPEG.obj
 0003:0000004c       _JPEGImageReader_skipPastImageID 1002304c     imageioJPEG.obj
 0003:00000050       _JPEGImageWriter_writeOutputDataID 10023050     imageioJPEG.obj
 0003:00000054       _JPEGImageWriter_warningOccurredID 10023054     imageioJPEG.obj
 0003:00000058       _JPEGImageWriter_warningWithMessageID 10023058     imageioJPEG.obj
 0003:0000005c       _JPEGImageWriter_writeMetadataID 1002305c     imageioJPEG.obj
 0003:00000060       _JPEGImageWriter_grabPixelsID 10023060     imageioJPEG.obj
 0003:00000064       _JPEGQTable_tableID        10023064     imageioJPEG.obj
 0003:00000068       _JPEGHuffmanTable_lengthsID 10023068     imageioJPEG.obj
 0003:0000006c       _JPEGHuffmanTable_valuesID 1002306c     imageioJPEG.obj
 0003:00000070       _sendHeaderInfoID          10023070     jpegdecoder.obj
 0003:00000074       _sendPixelsByteID          10023074     jpegdecoder.obj
 0003:00000078       _sendPixelsIntID           10023078     jpegdecoder.obj
 0003:0000007c       _InputStream_readID        1002307c     jpegdecoder.obj
 0003:00000080       _InputStream_availableID   10023080     jpegdecoder.obj
 0003:00000090       _GS_ExceptionRecord        10023090     MSVCRT:gs_report.obj
 0003:000000e0       _GS_ContextRecord          100230e0     MSVCRT:gs_report.obj
 0003:000003ac       ?__proc_attached@@3HA      100233ac     MSVCRT:dll_dllmain.obj
 0003:000003c0       ?is_initialized_as_dll@@3_NA 100233c0     MSVCRT:utility.obj
 0003:000003c1       ?module_local_atexit_table_initialized@@3_NA 100233c1     MSVCRT:utility.obj
 0003:000003c4       ?module_local_atexit_table@@3U_onexit_table_t@@A 100233c4     MSVCRT:utility.obj
 0003:000003d0       ?module_local_at_quick_exit_table@@3U_onexit_table_t@@A 100233d0     MSVCRT:utility.obj
 0004:00000060       $R000000                   10024060     jpeg.dll.res
